 gptsdk

 Timestamp is 4da293d4 (Mon Apr 11 17:38:28 2011)

 Preferred load address is 10000000

 Start         Length     Name                   Class
 0001:00000000 00000004H .CRT$XCA                CODE
 0001:00000004 00000004H .CRT$XCZ                CODE
 0001:00000008 00000004H .CRT$XIA                CODE
 0001:0000000c 00000004H .CRT$XIZ                CODE
 0001:00000010 00000004H .CRT$XPA                CODE
 0001:00000014 00000004H .CRT$XPZ                CODE
 0001:00000018 00000004H .CRT$XTA                CODE
 0001:0000001c 00000004H .CRT$XTZ                CODE
 0001:00000020 0000001cH .rdata                  CODE
 0001:0000003c 00000023H .rdata$debug            CODE
 0001:00000060 0000058cH .text                   CODE
 0001:000005ec 00000014H .idata$2                CODE
 0001:00000600 00000014H .idata$3                CODE
 0001:00000614 00000028H .idata$4                CODE
 0001:0000063c 0000000cH .idata$6                CODE
 0001:00000650 0000012bH .edata                  CODE
 0002:00000000 00000028H .idata$5                DATA
 0002:00000028 00000008H .data                   DATA
 0002:00000030 0000000cH .bss                    DATA
 0003:00000000 00000090H .pdata                  DATA

  Address         Publics by Value              Rva+Base       Lib:Object

 0000:00000000       ___safe_se_handler_table   00000000     <absolute>
 0000:00000000       ___safe_se_handler_count   00000000     <absolute>
 0001:00000000       __xc_a                     10001000     corelib0:crt0init.obj
 0001:00000004       __xc_z                     10001004     corelib0:crt0init.obj
 0001:00000008       __xi_a                     10001008     corelib0:crt0init.obj
 0001:0000000c       __xi_z                     1000100c     corelib0:crt0init.obj
 0001:00000010       __xp_a                     10001010     corelib0:crt0init.obj
 0001:00000014       __xp_z                     10001014     corelib0:crt0init.obj
 0001:00000018       __xt_a                     10001018     corelib0:crt0init.obj
 0001:0000001c       __xt_z                     1000101c     corelib0:crt0init.obj
 0001:00000060       GptOpenHandle              10001060 f   gptsdk_common_topaz_v1:gptsdk.obj
 0001:000000a0       GptCloseHandle             100010a0 f   gptsdk_common_topaz_v1:gptsdk.obj
 0001:000000c4       GptCreateTimerEvent        100010c4 f   gptsdk_common_topaz_v1:gptsdk.obj
 0001:00000140       GptReleaseTimerEvent       10001140 f   gptsdk_common_topaz_v1:gptsdk.obj
 0001:00000198       GptShowTimerSrc            10001198 f   gptsdk_common_topaz_v1:gptsdk.obj
 0001:000001dc       GptStart                   100011dc f   gptsdk_common_topaz_v1:gptsdk.obj
 0001:00000230       GptStop                    10001230 f   gptsdk_common_topaz_v1:gptsdk.obj
 0001:00000274       GptResume                  10001274 f   gptsdk_common_topaz_v1:gptsdk.obj
 0001:000002b8       GptUpdatePeriod            100012b8 f   gptsdk_common_topaz_v1:gptsdk.obj
 0001:00000304       GptGetCounterValue         10001304 f   gptsdk_common_topaz_v1:gptsdk.obj
 0001:00000350       DllEntry                   10001350 f   gptsdk_common_topaz_v1:gptsdk.obj
 0001:00000364       CreateFileW                10001364 f   coredll:COREDLL.dll
 0001:00000374       CloseHandle                10001374 f   coredll:COREDLL.dll
 0001:00000384       DeviceIoControl            10001384 f   coredll:COREDLL.dll
 0001:00000394       CreateEventW               10001394 f   coredll:COREDLL.dll
 0001:000003a4       DisableThreadLibraryCalls  100013a4 f   coredll:COREDLL.dll
 0001:000003b4       _DllEntryCRTStartup        100013b4 f   corelib0:pegdentry.obj
 0001:000004b8       _cexit                     100014b8 f   corelib0:cexit.obj
 0001:000004c8       _initterm                  100014c8 f   corelib0:crt0dat.obj
 0001:000004f4       _cinit                     100014f4 f   corelib0:crt0dat.obj
 0001:00000554       __security_init_cookie     10001554 f   corelib0:seccinit.obj
 0001:000005a0       __crt_ExitProcess          100015a0 f   corelib0:exitproc_proxy.obj
 0001:000005ac       wcslen                     100015ac f   corelib1:COREDLL.dll
 0001:000005bc       free                       100015bc f   corelib1:COREDLL.dll
 0001:000005cc       __security_gen_cookie2     100015cc f   corelib1:COREDLL.dll
 0001:000005dc       TerminateProcess           100015dc f   coredll:COREDLL.dll
 0001:000005ec       __IMPORT_DESCRIPTOR_COREDLL 100015ec     coredll:COREDLL.dll
 0001:00000600       __NULL_IMPORT_DESCRIPTOR   10001600     coredll:COREDLL.dll
 0002:00000000       __imp_CreateFileW          10002000     coredll:COREDLL.dll
 0002:00000004       __imp_CloseHandle          10002004     coredll:COREDLL.dll
 0002:00000008       __imp_DeviceIoControl      10002008     coredll:COREDLL.dll
 0002:0000000c       __imp_CreateEventW         1000200c     coredll:COREDLL.dll
 0002:00000010       __imp_DisableThreadLibraryCalls 10002010     coredll:COREDLL.dll
 0002:00000014       __imp_wcslen               10002014     corelib1:COREDLL.dll
 0002:00000018       __imp_free                 10002018     corelib1:COREDLL.dll
 0002:0000001c       __imp___security_gen_cookie2 1000201c     corelib1:COREDLL.dll
 0002:00000020       __imp_TerminateProcess     10002020     coredll:COREDLL.dll
 0002:00000024       \177COREDLL_NULL_THUNK_DATA 10002024     coredll:COREDLL.dll
 0002:00000028       __security_cookie          10002028     corelib0:seccinit.obj
 0002:0000002c       __security_cookie_complement 1000202c     corelib0:seccinit.obj
 0002:00000030       _exitflag                  10002030     corelib0:cexit.obj
 0002:00000034       __onexitend                10002034     <common>
 0002:00000038       __onexitbegin              10002038     <common>

 entry point at        0001:000003b4

 Static symbols

 0001:000003f8       doexit                     100013f8 f   corelib0:cexit.obj
